:100000000C9434000C9440000C943E000C943E0080
:100010000C943E000C943E000C943E000C943E0068
:100020000C943E000C943E000C943E000C943E0058
:100030000C943E000C943E000C943E000C943E0048
:100040000C943E000C943E000C943E000C943E0038
:100050000C943E000C943E000C943E000C943E0028
:100060000C943E000C943E0011241FBECFEFD4E050
:10007000DEBFCDBF0E94E9000C9429040C9400005F
:100080001FB6E0E0F1E079E10CC035E13A9511F1FD
:1000900049B14470D9F700000000000000000000E2
:1000A000000044D0589A49B15898447041937A95C9
:1000B00039F035E13A9571F049B14470D9F3E5CFA3
:1000C000E0E0F1E087882224882011F0239400C02A
:1000D00086803AC030E1371B21F5E0E0F1E0319154
:1000E0003323F9F4319131913323D9F4319133230E
:1000F000C1F431913323A9F43191332391F4319137
:10010000332379F431913323889409F00894E0E0A3
:10011000F1E031913081332311F018F410C008F070
:1001200009C01FBE189533941FBE189533E03A9549
:10013000F1F70895E9EBF2E078E114D0F2CFE1EDC8
:10014000F2E070E50FD0EDCF662019F4E9E1F1E0BF
:1001500002C0E9E6F1E0882011F070E501C070E42A
:1001600001D0E1CF31913323C9F40000529A4FE01E
:100170004A95F1F70000529842E04A95F1F77A95D6
:1001800089F7000000000000000000000000529A03
:1001900044E04A95F1F7000052980895529A44E0DD
:1001A0004A95F1F70000000052984CE04A95F1F7AB
:1001B000000000007A95B1F6000000000000000089
:1001C00000000000529A44E04A95F1F7000052986E
:1001D0000895002455244424439407EE08B900E30D
:1001E00007B90FEF05B900E004B90AEF0BB901E058
:1001F0000AB902E00093690001E00DBBB3D281D2DD
:100200008AD2D0D26624332468D244D05523E1F771
:100210007724C9EBD1E00A85002311F001E0702AB0
:100220000B85002311F002E0702A0E81002311F0EB
:1002300004E0702A0F81002311F008E0702A0C8579
:10024000002311F000E1702A0D85002311F000E277
:10025000702A0E85002311F000E4702A0F85002318
:1002600011F000E8702A12D078943320F1F3552071
:1002700051F44424439429F033241FD23320D1F77E
:1002800002C05524539406D03324EFCF00E8202E2B
:1002900017D00895552029F413D017E10AD21A95E2
:1002A000E9F701E003D0FF20C1F10895C9EBD1E0E7
:1002B00024D00993C9EBD1E009E0F02E80D2089553
:1002C000C9EBD1E003E019D000E8022529F000ECE9
:1002D00014D00BE112D004C000E80FD001E00DD023
:1002E0000EE0902E022D09D09A94E1F70993C9EB04
:1002F000D1E009E8F02E63D20895F02E00E8102F27
:100300001F2119930695D9F70895662019F4C9E6B7
:10031000D1E00895C9E1D1E00895172D107F00E1E3
:100320000127002311F4A0D013C000E2012700230D
:1003300011F4D7D00DC000E40127002311F40ED131
:1003400007C000E80127002311F44AD101C02ED0D4
:10035000DCDF0985FF24002309F0F09418E0E09623
:10036000F9921A95E9F7D1DF0A85FF24002309F0F5
:10037000F09418E0E896F9921A95E9F7A9EBB1E044
:1003800050966BD172FE79D110E82127BEDF6096BE
:100390006DD1A9EBB1E0589660D172FE6ED110E834
:1003A0002127B3DF689662D160940895A9EBB1E08C
:1003B000ACDF0D910F830D910E830D9170FE0987B7
:1003C00070FC0B870D910B830D910C870D910D87A0
:1003D0000D910F870D910E8712960D9170FE0B8770
:1003E00070FC09870D910A8771FE09C0A9EBB1E085
:1003F0001E960C910C831E971F960C910D83A9EBF2
:10040000B1E083DF1C960C91002341F4A9EBB1E02D
:100410001D960C91002321F40FE703C00FEF01C0DC
:1004200000E010E8A896F12EF022F9921695D9F77F
:1004300071FC19C0A9EBB1E068DF1E960C91002396
:1004400041F4A9EBB1E01F960C91002321F40FE7D2
:1004500003C000E001C00FEF10E8A096F12EF022DB
:10046000F9921695D9F70895A9EBB1E04EDF0D91F9
:100470000F830D910E830D9109870D910B830D91C3
:100480000C870D910D870D910F870D910E87129698
:100490000D910A870D910B870D910D910D830D9193
:1004A0000C830FE7A9EBB1E01C961C91112309F016
:1004B0000FEF10E8A896F12EF022F9921695D9F7D1
:1004C0000FE723DFA9EBB1E01F961C91112309F080
:1004D0000FEF10E8A096F12EF022F9921695D9F7B9
:1004E0000895A9EBB1E011DF0D910F830D910E83FB
:1004F0000D9109870D910B830D910A870D910D8741
:100500000D910F870D910E8712960D910C870D910D
:100510000B870D910D910D830D910C830FE7A9EBC6
:10052000B1E01C961C91112309F00FEF10E8A8967A
:10053000F12EF022F9921695D9F70FE7E6DEA9EB36
:10054000B1E01F961C91112309F00FEF10E8A0965F
:10055000F12EF022F9921695D9F70895A9EBB1E0A2
:10056000D4DE0D910F830D910E830D9109870D91AE
:100570000B830D910C870D910D870D910F870D91B8
:100580000E8712960D910A870D910B870D910D9193
:100590000D830FE7A9EBB1E01C961C91112309F024
:1005A0000FEF10E8A896F12EF022F9921695D9F7E0
:1005B0000FE7ABDEA9EBB1E01E961C91112309F009
:1005C00000E0A9EBB1E01F961C91112309F00FEF99
:1005D00010E8A096F12EF022F9921695D9F7089519
:1005E000A9EBB1E092DE0D910F830D910E830D9179
:1005F0000A870D910B830D910C870D910D870D913D
:100600000F870D910E8712960D9109870D910B871B
:100610000D910D910C830D910D830FE7A9EBB1E0C6
:100620001C961C91112309F00FEF10E8A896F12EEB
:10063000F022F9921695D9F70FE767DEA9EBB1E042
:100640001F961C91112309F00FEF10E8A096F12ED0
:10065000F022F9921695D9F70895222710E80D9106
:10066000002309F0212B1695D1F7089510E8F12EFB
:10067000F222F9921695D9F7089573FE04C0022F5D
:100680000595020F07C0022F05950595102F1595AA
:10069000020F010F00231AF022233AF009C022238F
:1006A0000AF406C00FE7202F04C000E8202F01C085
:1006B000202F0EE10A95F1F708951F931AE00FEF2E
:1006C00000000000000000000000000000000A958B
:1006D000B9F71A95A1F71F9108951F9317E60FEF29
:1006E00000000000000000000000000000000A956B
:1006F000B9F700000000000000001A9581F71F9173
:10070000089531E0E9EBF2E034963083339630839C
:100710003B963083089531E0E1EDF2E03896308386
:1007200038963083369631933083329631933193B5
:1007300031933083329630833296308337963083CC
:10074000329631933193319331933193308335968F
:10075000308332963193308335963083339631939C
:10076000308308954427E9EBF2E038E141933A956C
:10077000E9F7E1EDF2E030E541933A95E9F7E9E593
:10078000F1E0C9EAD1E030E1419349933A95E1F7CC
:10079000E9E5F1E0C9EAD1E00FEF078307870F83AE
:1007A0000F870895A9E6B1E0E9E1F1E0C1EDD2E0FB
:1007B00000E4499141934D930A95D9F70895099121
:1007C000002369F400003B9A1FE01A95F1F700003E
:1007D0003B9812E01A95F1F7FA9489F70EC03B9A0C
:1007E00014E01A95F1F7000000003B981CE01A9500
:1007F000F1F700000000FA9411F755275095C9EB66
:10080000D1E021E205E10A95F9F016B11870D9F7A7
:1008100000000000000000000000000011D0589A05
:1008200016B15898187019932A9539F005E10A9570
:1008300059F016B11870D9F3E5CFFF245527089564
:1008400003E00A95F1F70895FF24F3945527509596
:060850000895F894FFCFAB
:00000001FF
